:107000000C9468380C94A0380C9485380C9485380E
:107010000C9485380C9485380C9485380C948538FC
:107020000C9485380C9485380C9485380C948538EC
:107030000C9485380C9485380C9485380C948538DC
:107040000C9485380C9485380C9485380C948538CC
:107050000C9485380403090412036F006200640075
:10706000650076002E00610074001003480049009E
:10707000440042006F006F00740012011001000014
:107080000008C016DF05010101020001090222000B
:107090000101008032090400000103000000092101
:1070A00001010001222100070581030800C8060034
:1070B000FF0901A101150026FF007508850195064D
:1070C0000900B20201850295830900B20201C000E5
:1070D00011241FBECFE5D8E0DEBFCDBF10E0A0E693
:1070E000B0E0E6E8F9E702C005900D92AA36B107D4
:1070F000D9F710E0AAE6B0E001C01D92A43AB107AA
:10710000E1F70E94243C0C94C13C0C940038A82F59
:10711000B92F80E090E041E050EA609530E009C08E
:107120002D9182279795879510F084279527305EBB
:10713000C8F36F5FA8F30895EADF8D939D930895D8
:10714000CF93CFB7CF93C395839BE9F7839B09C0B8
:10715000839B07C0839B05C0839B03C0839B01C0A7
:10716000A3C0DF93C0918700DD27C257DF4F839B09
:1071700002C0DF91EBCF2F930F931F9300B32FEF3C
:1071800003FB20F94F933F9310B34FEF012703FB0D
:1071900021F93BE031C04E7F012F10B3216028C0A0
:1071A000102F4D7F2260000000B329C04B7F246068
:1071B000012F000010B32BC010B3477F28602AC0F6
:1071C0004F7E00B320612CC04F7D10B320622FC0D2
:1071D0004F7B00B3206432C0422700B349934FEF86
:1071E0000000102713FB20F910B31C70C9F1297F90
:1071F00091F2012703FB21F900B3237F89F231507B
:1072000058F1102713FB22F910B3277E79F20127DA
:1072100003FB23F92F7C81F200B3102713FB24F921
:107220002F7971F200C010B3012703FB25F92F73EA
:1072300059F200C000B3102713FB26F9223040F2A8
:1072400000C010B3012703FB27F9243028F64F773D
:10725000206810B30000F9CF10E41ABF002719C04E
:107260003B503195C31BD04010E41ABF0881033C4A
:10727000F9F00B34E9F0209185001981110F1213F8
:10728000EDCF4A81441F093641F10D3211F0013E24
:1072900029F700938C003F914F911F910F912F91EF
:1072A000DF91CAB7C6FD4FCFCF91CFBFCF91189511
:1072B00020918C00222379F310918A00112321F56B
:1072C000343022F130938A00209386001091870099
:1072D0003BE0311B3093870019C000918A000130D8
:1072E0009CF40AE54F7081F43091600034FD10C0C9
:1072F00000936000C9E7D0E00FC02795A8F4515073
:10730000A9F4220F0000F9CF4AE503C042ED01C005
:10731000432FC4E1D0E032E011B31C60939A11BB5B
:1073200002B320E41CE05F93012756E002BB2795DF
:1073300020F4515021F4220FF9CF012756E000002C
:107340003B5A02BBD0F2279528F4515029F4220F62
:107350000000F9CF012756E0279502BB20F45150D9
:1073600021F4220FF9CF012756E02991332302BBE4
:1073700021F6037F10918B00110FC651D04002BB44
:1073800011F01093850010E41ABF086011B3137F49
:10739000402F437F5F9100C000C002BB11BB42BBC6
:1073A0007ACF80916D00882309F452C088EB9BE06E
:1073B0000197F1F780916A008F5F80936A00909146
:1073C0006100891709F042C010926A0080916B0039
:1073D000833011F1843028F4813089F08230A0F4B8
:1073E00007C0853019F18530E0F0863069F523C09B
:1073F00082B38C7A82BB81E080936B0021C082B320
:10740000836582BB82E004C082B38C7A82BB83E056
:1074100080936B008FE715C082B3836582BB84E0E5
:10742000F7CF82B38C7A82BB85E0F2CF82B38365DB
:1074300082BB86E0EDCF82B38C7A82BB10926B0068
:107440008FEF8093610002C010926B0081E008957D
:1074500029B3237040916E000DC089B330E090E0F5
:10746000837090702817390711F040E001C04F5F1A
:1074700029B32370463088F32093720040936E0046
:10748000233018F481E080936D0080916D000895A1
:1074900085B7826085BF8BB780648BBF0895F894F1
:1074A00081E180935700E8951BBE15BE81E08BBF3C
:1074B0001BBE8B9AE0917700F0917800099521E04E
:1074C00020936C00FC018181893069F482818230D3
:1074D00029F4209375002093840003C082E08093F8
:1074E00084008FEF0895813011F080E0089582E6E6
:1074F00090E0909389008093880087E00895CF936F
:10750000DF93DC01C0917000D0917100413051F4E3
:1075100010926F001196CC9111971296DC911297F0
:107520001496645030916F00360F30936F00AE01A7
:107530004F7751F4F89483E0FE0180935700E8956B
:10754000789407B600FCFDCFF894AE018D919C9124
:10755000119721E0FE010C0120935700E8951124BA
:1075600078942296FE01EF7751F4F89485E0FA01C1
:1075700080935700E895789407B600FCFDCF6250E1
:1075800011F01296D4CFD0937100C0937000832F66
:107590008078DF91CF910895CF93DF93FC018091A4
:1075A0008400813071F480917500813029F410924B
:1075B0007500CF0141E002C0CF0140E00E947F3A58
:1075C0002FC0823061F58181813011F40E944F3AE1
:1075D0008F3F21F484E090E06FEF19C08E3F91F46B
:1075E00082B3836582BBC0E0D0E0CE016FEF0E9422
:1075F000B43C219684E0C030D807B9F782B38C7AC6
:1076000082BB0BC08D3F31F48281938164810E94E3
:10761000B43C03C081E0809376001092840081E046
:10762000DF91CF9108951F93CF93DF9360918A00EC
:10763000635067FDBAC080918700CCE0D0E0C81BE2
:10764000D109C257DF4F809186008D3209F09AC070
:10765000683009F0A8C083EC809379008AE58093B4
:107660006000109274008881807641F0CE010E9403
:107670005F3A282F8F3F09F474C07AC09A81109224
:1076800082008981882321F41092830022E062C065
:10769000853019F490938B005CC0863009F04AC0A5
:1076A0008B81813019F48AE790E71BC0823041F466
:1076B0008CE890E7909389008093880022E236C09E
:1076C0008330F9F48A81882341F484E590E790932C
:1076D00089008093880024E029C0813041F488E546
:1076E00090E7909389008093880022E11FC0823048
:1076F000E1F48AE690E7909389008093880020E186
:1077000015C0813241F48EE990E79093890080930F
:10771000880029E00BC0823241F48EEA90E7909312
:1077200089008093880021E201C020E080E48093FA
:1077300074001EC0883021F421E08DE890E00CC078
:10774000893019F490938D0004C08A3011F421E03F
:1077500001C020E082E890E0909389008093880047
:1077600007C0888187FD2E8180E88093740006C061
:107770008F81882319F48E81821708F0822F8093DD
:10778000690011C08091740087FF0DC0CE010E9476
:10779000CC3A8F3F21F48EE18093600004C08823AF
:1077A00011F01092690010928A008091600084FFAD
:1077B0003DC0809169008F3FC9F1182F893008F0D2
:1077C00018E0811B809369008091790098E88927EF
:1077D000809379001123E1F0E0918800F091890015
:1077E0008091740086FF09C0912FAAE7B0E08491D0
:1077F0008D9331969150D9F707C0912FAAE7B0E049
:1078000081918D939150E1F7F0938900E093880086
:107810008AE790E0612F0E949C38612F6C5F6C308A
:1078200019F08FEF809369006093600094E180B35A
:107830008C7031F49150D9F710928B001092850022
:10784000DF91CF911F91089581B3836581BB82B38E
:107850008C7A82BB8D98959A8AB38C7F8ABB8BB3C6
:1078600083608BBBB89AC09881E090E00E949B3CFB
:1078700080937300882349F481E080936D0081E058
:1078800090E06FEF0E94B43C08C0E0E0F0E0E491CB
:10789000EF3F19F481E080936D000E94D139882375
:1078A00009F447C081E08BBF82E08BBF0E94483A59
:1078B00088E991E00E949B3C882349F48B9A20E060
:1078C000A89588EB9BE00197F1F72150C9F78B98B9
:1078D00078940FEF10E0C0E0D0E080916C00882336
:1078E000B9F487E2C131D80714F4219611C0F89495
:1078F00081E090E060E00E94A33C8B9A28E088E160
:1079000090E00FB6F894A89581BD0FBE21BDFFCFC2
:10791000A8950E94133B80917600882331F00023C4
:1079200019F4115011F405C001500E94D139882377
:10793000A1F60E944F3AE199FECF9FBB8EBBE09A21
:1079400099278DB30895262FE199FECF9FBB8EBB5B
:10795000E09A01970DB2021631F02DBB0FB6F894E4
:10796000E29AE19A0FBE0895262FE199FECF9FBBC0
:107970008EBB2DBB0FB6F894E29AE19A0FBE01962A
:067980000895F894FFCF0A
:0A7986005A7F01800000800000FF1E
:040000030000700089
:00000001FF
